 mouhid

 Timestamp is 4da293b9 (Mon Apr 11 17:38:01 2011)

 Preferred load address is 10000000

 Start         Length     Name                   Class
 0001:00000000 00000004H .CRT$XCA                CODE
 0001:00000004 00000004H .CRT$XCZ                CODE
 0001:00000008 00000004H .CRT$XIA                CODE
 0001:0000000c 00000004H .CRT$XIZ                CODE
 0001:00000010 00000004H .CRT$XPA                CODE
 0001:00000014 00000004H .CRT$XPZ                CODE
 0001:00000018 00000004H .CRT$XTA                CODE
 0001:0000001c 00000004H .CRT$XTZ                CODE
 0001:00000020 00000090H .rdata                  CODE
 0001:000000b0 00000023H .rdata$debug            CODE
 0001:000000d4 00000aa4H .text                   CODE
 0001:00000b78 00000004H .xdata                  CODE
 0001:00000b7c 00000028H .idata$2                CODE
 0001:00000ba4 00000014H .idata$3                CODE
 0001:00000bb8 0000005cH .idata$4                CODE
 0001:00000c14 000000aaH .idata$6                CODE
 0001:00000cc0 0000006eH .edata                  CODE
 0002:00000000 0000005cH .idata$5                DATA
 0002:0000005c 00000008H .data                   DATA
 0002:00000064 00000018H .bss                    DATA
 0003:00000000 00000088H .pdata                  DATA

  Address         Publics by Value              Rva+Base       Lib:Object

 0000:00000000       ___safe_se_handler_table   00000000     <absolute>
 0000:00000000       ___safe_se_handler_count   00000000     <absolute>
 0001:00000000       __xc_a                     10001000     corelib0:crt0init.obj
 0001:00000004       __xc_z                     10001004     corelib0:crt0init.obj
 0001:00000008       __xi_a                     10001008     corelib0:crt0init.obj
 0001:0000000c       __xi_z                     1000100c     corelib0:crt0init.obj
 0001:00000010       __xp_a                     10001010     corelib0:crt0init.obj
 0001:00000014       __xp_z                     10001014     corelib0:crt0init.obj
 0001:00000018       __xt_a                     10001018     corelib0:crt0init.obj
 0001:0000001c       __xt_z                     1000101c     corelib0:crt0init.obj
 0001:0000005c       ??_C@_1CG@NNBNONKD@?$AAM?$AAo?$AAu?$AAs?$AAe?$AAA?$AAt?$AAt?$AAa?$AAc?$AAh?$AAe?$AAd?$AAE?$AAv?$AAe?$AAn?$AAt?$AA?$AA@ 1000105c     mouhid.obj
 0001:00000084       ??_C@_1CG@JHDABJCF@?$AAM?$AAo?$AAu?$AAs?$AAe?$AAD?$AAe?$AAt?$AAa?$AAc?$AAh?$AAe?$AAd?$AAE?$AAv?$AAe?$AAn?$AAt?$AA?$AA@ 10001084     mouhid.obj
 0001:000000d4       DllEntry                   100010d4 f   mouhid.obj
 0001:0000016c       HIDDeviceNotifications     1000116c f   mouhid.obj
 0001:000005b0       HIDDeviceAttach            100015b0 f   mouhid.obj
 0001:00000774       HidP_GetSpecificValueCaps  10001774 f   hidparse:HIDPARSE.dll
 0001:00000784       HidP_GetScaledUsageValue   10001784 f   hidparse:HIDPARSE.dll
 0001:00000794       HidP_UsageListDifference   10001794 f   hidparse:HIDPARSE.dll
 0001:000007a4       HidP_GetUsages             100017a4 f   hidparse:HIDPARSE.dll
 0001:000007b4       HidP_MaxUsageListLength    100017b4 f   hidparse:HIDPARSE.dll
 0001:000007c4       HidP_GetCaps               100017c4 f   hidparse:HIDPARSE.dll
 0001:000007d4       DriverMouseHookInitialize  100017d4 f   MouHidStd:StandardMouse.obj
 0001:000007dc       DriverMouseHook            100017dc f   MouHidStd:StandardMouse.obj
 0001:000007e4       EventModify                100017e4 f   coredll:COREDLL.dll
 0001:000007f4       CloseHandle                100017f4 f   coredll:COREDLL.dll
 0001:00000804       CreateEventW               10001804 f   coredll:COREDLL.dll
 0001:00000814       DisableThreadLibraryCalls  10001814 f   coredll:COREDLL.dll
 0001:00000824       LocalAlloc                 10001824 f   coredll:COREDLL.dll
 0001:00000834       mouse_event                10001834 f   coredll:COREDLL.dll
 0001:00000844       LocalFree                  10001844 f   coredll:COREDLL.dll
 0001:00000854       WaitForSingleObject        10001854 f   coredll:COREDLL.dll
 0001:00000864       SetThreadPriority          10001864 f   coredll:COREDLL.dll
 0001:00000874       CreateThread               10001874 f   coredll:COREDLL.dll
 0001:00000884       _DllEntryCRTStartup        10001884 f   corelib0:pegdentry.obj
 0001:000008c8       __GSHandlerCheckCommon     100018c8 f   corelib0:gshandler.obj
 0001:00000900       __GSHandlerCheck           10001900 f   corelib0:gshandler.obj
 0001:00000920       __security_init_cookie     10001920 f   corelib0:seccinit.obj
 0001:0000096c       __security_check_cookie    1000196c f   corelib0:armsecgs.obj
 0001:0000097c       __gsfailure                1000197c     corelib0:armsecgs.obj
 0001:00000a80       _cexit                     10001a80 f   corelib0:cexit.obj
 0001:00000a90       _initterm                  10001a90 f   corelib0:crt0dat.obj
 0001:00000abc       _cinit                     10001abc f   corelib0:crt0dat.obj
 0001:00000b1c       __crt_ExitProcess          10001b1c f   corelib0:exitproc_proxy.obj
 0001:00000b28       memcpy                     10001b28 f   corelib1:COREDLL.dll
 0001:00000b38       __security_gen_cookie2     10001b38 f   corelib1:COREDLL.dll
 0001:00000b48       __report_gsfailure         10001b48 f   corelib1:COREDLL.dll
 0001:00000b58       free                       10001b58 f   corelib1:COREDLL.dll
 0001:00000b68       TerminateProcess           10001b68 f   coredll:COREDLL.dll
 0001:00000b7c       __IMPORT_DESCRIPTOR_HIDPARSE 10001b7c     hidparse:HIDPARSE.dll
 0001:00000b90       __IMPORT_DESCRIPTOR_COREDLL 10001b90     coredll:COREDLL.dll
 0001:00000ba4       __NULL_IMPORT_DESCRIPTOR   10001ba4     hidparse:HIDPARSE.dll
 0002:00000000       __imp_LocalFree            10002000     coredll:COREDLL.dll
 0002:00000004       __imp_free                 10002004     corelib1:COREDLL.dll
 0002:00000008       __imp___report_gsfailure   10002008     corelib1:COREDLL.dll
 0002:0000000c       __imp___security_gen_cookie2 1000200c     corelib1:COREDLL.dll
 0002:00000010       __imp_EventModify          10002010     coredll:COREDLL.dll
 0002:00000014       __imp_CloseHandle          10002014     coredll:COREDLL.dll
 0002:00000018       __imp_CreateEventW         10002018     coredll:COREDLL.dll
 0002:0000001c       __imp_DisableThreadLibraryCalls 1000201c     coredll:COREDLL.dll
 0002:00000020       __imp_LocalAlloc           10002020     coredll:COREDLL.dll
 0002:00000024       __imp_mouse_event          10002024     coredll:COREDLL.dll
 0002:00000028       __imp_TerminateProcess     10002028     coredll:COREDLL.dll
 0002:0000002c       __imp_WaitForSingleObject  1000202c     coredll:COREDLL.dll
 0002:00000030       __imp_SetThreadPriority    10002030     coredll:COREDLL.dll
 0002:00000034       __imp_CreateThread         10002034     coredll:COREDLL.dll
 0002:00000038       __imp_memcpy               10002038     corelib1:COREDLL.dll
 0002:0000003c       \177COREDLL_NULL_THUNK_DATA 1000203c     coredll:COREDLL.dll
 0002:00000040       __imp_HidP_GetCaps         10002040     hidparse:HIDPARSE.dll
 0002:00000044       __imp_HidP_MaxUsageListLength 10002044     hidparse:HIDPARSE.dll
 0002:00000048       __imp_HidP_GetUsages       10002048     hidparse:HIDPARSE.dll
 0002:0000004c       __imp_HidP_UsageListDifference 1000204c     hidparse:HIDPARSE.dll
 0002:00000050       __imp_HidP_GetScaledUsageValue 10002050     hidparse:HIDPARSE.dll
 0002:00000054       __imp_HidP_GetSpecificValueCaps 10002054     hidparse:HIDPARSE.dll
 0002:00000058       \177HIDPARSE_NULL_THUNK_DATA 10002058     hidparse:HIDPARSE.dll
 0002:0000005c       __security_cookie          1000205c     corelib0:seccinit.obj
 0002:00000060       __security_cookie_complement 10002060     corelib0:seccinit.obj
 0002:00000070       _exitflag                  10002070     corelib0:cexit.obj
 0002:00000074       __onexitend                10002074     <common>
 0002:00000078       __onexitbegin              10002078     <common>

 entry point at        0001:00000884

 Static symbols

 0001:0000027c       ?ProcessMouseReport@@YAXPAU_HID_MOUSE@@PADK@Z 1000127c f   mouhid.obj
 0001:000004f8       ?MouseThreadProc@@YAKPAX@Z 100014f8 f   mouhid.obj
 0001:000009c0       doexit                     100019c0 f   corelib0:cexit.obj
